:020000040000FA
:060000000219FD020310CD
:030013000204FFE5
:03001B0002008D53
:03002B000202D5F9
:03005B0002050E8D
:030073000202FD89
:100080000406080C10182030406080A0C0C2AFC227
:10009000A853E6EFC28E856B8BC0D0D2D3C0E0C030
:1000A000F0C2CAA8CCA9CDD2CAD2AF758A00C3E823
:1000B000956CF8E9956DF9C3E913F9E813F8E5666D
:1000C0006007C3E913F9E813F8E97025E8956E4075
:1000D00020956E501CE582B410177C007B007A00DE
:1000E0007908900000A86AE5667004C3E813F80177
:1000F000FA900000D2A8D2AA61BAE0FDC39CC398CE
:1001000040EF98EB33FB0582E0FCC39DC39840E1D0
:1001100098EB33FB0582E0FDC39CC39840D398EB7A
:1001200033FB0582E0FCC39DC39840C598EB33FBCD
:100130000582E0FDC39CC39840B798EB33FB058272
:10014000E0FCC39DC39840A998EB33FB0582E0FD1A
:10015000C39CC398409B98EB33FB0582E0FCC39D96
:10016000C398408D98EB33FB05822175900000D237
:10017000A8D2AA61BAE0FDC39CC39840EF98EA33C5
:10018000FA0582E0FCC39DC39840E198EA33FA0582
:1001900082E0FDC39CC39840D398EA33FA0582E01D
:1001A000FCC39DC39840C598EA33FA0582E0FDC3BD
:1001B0009CC39840B798EA33FA0582E0FCC39DC31C
:1001C0009840A998EA33FA0582E0FDC39CC39840A1
:1001D0009B98EA33FA0582E0FCC39DC398408D9852
:1001E000EA33FA0582EBC46B6A54F0F9EAC454F0BE
:1001F000C3996009900000D2A8D2AA61BAEBF4C4F6
:1002000054F0F9EAF4C4540F49FAEBF4C4540FFB68
:10021000C3EAF99460FAEB9400FB5020C3E97B0039
:100220007A0079006016C3135006F9C39552600A2C
:10023000E9F552755300790080020553303A27C31F
:10024000EA94D0F8EB9407F9400BE8FAE9FB203583
:1002500009D235415A303502C235203902B235C390
:10026000EA33FAEB33FBEB2B3B3BF9C3EB13FBEA33
:1002700013FAEA29FAEB3400FB30E3047AFF7BFF40
:10028000E5255403601B202A18E55D33F9EB700760
:10029000C3E99A4002E9FAE53CC4332AFAEB340098
:1002A000FBC3EA33C4540FF8EB33C454F048F8707E
:1002B00005EA60027801C3EB13FBEA13FA90000031
:1002C000D2A8D2AAE52260021522819E900000D217
:1002D000A8D2AA61BAC0D0C0E0C2CF0541E5236070
:1002E000021523C3E554600575550041F8E5552412
:1002F00001F55550037555FFD0E0D0D032C2AF5351
:10030000E67F7592FA7593FFC22053917FD2AF3288
:10031000C0E0E58A303408856B8BF0A3D0E032D0A2
:10032000E0C2AF53E6EFC0D0C0E0C0F0D2D3D2AF4E
:100330005388EFA88AA98C758A00758C00438810B1
:1003400030331FE8C4540FFAE9C454F04AFAC31317
:100350002AFAC3E833F8E933F9E82AFAE93403FB67
:1003600061AB30320FC3E833E933FAE82AFAE934F3
:1003700000FB61AB303115E875F056A4AAF0E975C1
:10038000F056A42AFAC5F03400FB61ABE875F02BF7
:10039000A4AAF0E975F02BA42AFAC5F03400C3131F
:1003A000FBEA13FAC3EB13FBEA13FAC3EB9409500D
:1003B00009C3EA949AEB940350160522E5227002D1
:1003C0001522C3E5229432500281F275540081F562
:1003D000E522600215223036067C007D0461EAAC1D
:1003E00031AD32303A04AC33AD34C3EA9CFAEB9D04
:1003F000FB9208AE60AF61303A425007203509D217
:10040000358108303502C235303504AE62AF632025
:100410003902B235C3EA33FAEB33FBA208500AEAD9
:10042000F42401FAEBF43400FBC3EA9428FAEB94C9
:1004300000FB501478007A007B008148A208500825
:1004400078007A007B00819EE52554036019202AFC
:1004500016E55DF9EB7007C3E99A4002E9FAE53C5D
:10046000C42AFAEB3400FBEA8EF0A4F9AAF0EB8E72
:10047000F0A42AFAC5F03400FBC3EB13FDEA13F82D
:100480000FEF146004C3E833F8C3E933EA33FAEB3F
:1004900033FBDFEDEB30E20678FF7AFF7B03885415
:1004A000D230E86003755500C3E55BFC955C400203
:1004B000AC5CC3EC95545008EC75F004A4FAABF0B6
:1004C000EAF4F8EBF45403F9C3E8941EFAE9940053
:1004D000FB50047A007B00885689578A588B5975DF
:1004E000230AD0F0D0E0D0D053F7DF43F74043E603
:1004F000103275230AD0F0D0E0D0D043E61032C2DB
:10050000AAD28EC2CA85CC6C85CD6DD2CA32C2AF9A
:10051000C0D0C0E0D2D3A8F9E55A30E10AE5FA200C
:10052000E13520E032A12FE5FA30E12B20E028C3AD
:10053000E55713F8E55613F5FB88FCC3E55913F8A6
:10054000E55813F5E988EA85575A53F7BFD2A83022
:100550003402D2AA53E6EF53F7DFD0E0D0D0D2AFC7
:10056000327901801479038010790A800C791E8019
:10057000087964800479C880007817E4D5E0FDD854
:10058000FAD9F62278FF20282879A1E76023E548E8
:10059000601F74FF8548F084853FF030290375F0B3
:1005A00005A4F8C5F0600278FFC3E8955D5002A885
:1005B0005D885C22C3E54794E4E5489400E55C501F
:1005C0000314A1C5046002F55C2275E89022055E63
:1005D000C3E55E9408405330EDF4A8BDA9BE755E36
:1005E00000E9FA79A0E76041EA7006E55F601880EB
:1005F0000CC3E8955F600EE55F5005600A14800744
:100600000460FA8002E55FF55FC39569401B755B86
:10061000C0C394044013755B80C39404400B755BA6
:1006200040C394044003755B0022E55B2410500234
:1006300074FFF55B22743279A687F0A4C5F0A2F7A7
:1006400033F55D227547007548F022C2AFC2CAA8D3
:10065000CCA9CDAA4130CF010AD2CAD2AFAB42ACAD
:100660004388428943C3E89BF8E99C202808F93075
:100670002C02E15BC1B4AD448A44F9EA9DFA6006FC
:1006800078FF79FFC199AE45AF468B458C46A842AD
:10069000A943C3E89EF8E99FF9C3E54813FBE54782
:1006A00013FAE82AF547E93BF54850067547FF7508
:1006B00048FFE101AA47AB48AC47AD487E047F0242
:1006C000C3EB9404400D1E1FC3EB94084005202982
:1006D000021E1FC3ED13FDEC13FCDEF7C3EA9CFA08
:1006E000EB9DFBEF6009C3E913F9E813F8DFF7EAC4
:1006F00028FAEB39FB8A478B4850067BFF8B478BE8
:1007000048C3EB94025002D22C3028047F03E12C22
:100710007892E6FFC3E53D948240110FC3E53D9416
:10072000A040010FC3EF940640027F057E02E5481A
:10073000C4540FF9E548C454F0F8E547C4540F28F1
:10074000F8C3E89EFAE99400FB4009C3EA9401EB80
:10075000940050047A01E4FB0207A7AA47AB48EBD8
:10076000C4FEEAC4540F4EFCC3EA9CFAEB9400FBAF
:10077000C3E813C313F8EA28FAEB3400FB8A478B6B
:1007800048C3EB94024002C22C7802EBC4FE7B000B
:10079000EAC4540F4EFAC3EA98FA4005C3940150D4
:1007A000027A017892E6FF302002E1A7854E928519
:1007B0004F93D22043E680C3E49AF8E49BF9302CAF
:1007C00003020835E8FAE9FBD3E913FDE813FC88D6
:1007D0004E894FC3EF94036038EF20E00CE82CF80B
:1007E000E93DF9ECFAEDFB8013E828F8E939F9C3A3
:1007F000E82401F8E93400F97AFF7BFFC3EF9403A2
:10080000400F8A508B51884A894B8C4C8D4D020881
:100810006A885089518A4A8B4B8C4C8D4D302812F6
:100820007550F07551FF754CF0754DFF754EF075B4
:100830004FFF02086AE8FAD3E813FC884EC3EF942E
:10084000036021EF20E007E82CF8ECFA0155E828D6
:100850002401F87AFFC3EF940340098A50884A8C38
:100860004C02086A88508A4A8C4C302002016A7512
:100870003A02D22043E680E52554036034A847A914
:1008800048C3E913F9E813F8C3E913F9E813F8309A
:100890002804E92440F9C2AF53E67F759100C3E410
:1008A00098F594E499F595759104D22043E680D2A9
:1008B000AF22D221754900752000302B03752040EE
:1008C00001D0D221754900752040302B03752000DE
:1008D00078017901202C20E52554036002C221799A
:1008E00014E548C313700104F8C39414400278144B
:1008F000302804781B791B202010E549600C302833
:1009000003D53A04D222217711720549E59B544060
:10091000B52002216130280908C3E8994001180177
:10092000F720210A08C3E899400201D001F7C2214B
:1009300053E67F759100302C117594007595F8750C
:100940009104D22043E6800208D0E5487EFFC333FD
:100950004005C3334001FEC3E49E759400F5952124
:100960003FC3E5399401500201D030210201D0D8B3
:1009700002217501F7C222C2AF53E67F759100854F
:100980005094855195759104854A92854B93D22058
:1009900043E680D2AFE525540360072029020539DC
:1009A000801030220D202B0A20210715811581028D
:1009B00013782278003021027801E53D75F007A414
:1009C000F9E5F028F5F0E9A2F013A2F113A2F21371
:1009D000F53DC394785003753D78C3E53D953E40A1
:1009E00009C290C292C29475D57F30200221EA8557
:1009F0004C92854D93D22043E68022203810C2AF1E
:100A0000C293D29175D54FD2AF759F2041CBC2AF63
:100A1000C293D29575D57CD2AF759F2041CB20383B
:100A200010C2AFC29475D573D291D2AF759F3041C9
:100A3000CBC2AFC29075D573D295D2AF759F10411E
:100A4000CB203810C2AFC291D29575D573D2AF7595
:100A50009F108077C2AFC295D29175D573D2AF7512
:100A60009F308067203810C2AFC29275D57CD29576
:100A7000D2AF759F208054C2AFC29275D54FD2912C
:100A8000D2AF759F208044203810C2AFC295D29358
:100A900075D57CD2AF759F308031C2AFC291D293F1
:100AA00075D54FD2AF759F108021203810C2AFC2CC
:100AB0009075D54FD293D2AF759F10800EC2AFC242
:100AC0009475D57CD293D2AF759F30227A147B78FF
:100AD00080127A107B8C800C7A0D7BB480067A0BA6
:100AE0007BC88000E564D5E001227902E4C293D599
:100AF000E0FDD292D5E0FDC292D5E0FDD293D5E0E3
:100B0000FDE920E002D29030E002D294E564D5E025
:100B1000FDE920E002C29030E002C2947496D5E074
:100B2000FDD9C9EAF8D5E0FDD8FBDBB8C29322C2F3
:100B300090C292C294C291C293C29575D57F227819
:100B40008076FF0876FF0876FF0876FF0876FF08B4
:100B500076FF0876090876FF087601788C7601081A
:100B600076FF0876FF0876FF0876FF0876FF08769E
:100B7000030876FF0876FF0876FF0876250876D00A
:100B80000876280876500876040876FF087602086A
:100B900076FF08767A0876FF0876070876010876E9
:100BA000FF0876FF08760008760022FA75F00CA49C
:100BB000ABF0EAC333F8740133F9E8C333F8E9332F
:100BC000F9E8C32BF8E93400F9227888E6C39403E6
:100BD000D23A5002C23AC238E630E102D238A238E4
:100BE00092397886E6149000809378A6F67886E6A7
:100BF000F53FC394025003753F02789CE6753EFFB3
:100C0000B40203753EA0B40303753E8278A0E6F8F3
:100C1000600674282409D8FCF5697896E671AB88DB
:100C2000318932789EE671AB883389347897E671E2
:100C3000AB88358936712F223036117A007B007CE3
:100C4000FF7D007E00919E8B618A6022303A22787F
:100C500096E6FA7B00789EE6FC7D00C3EA33FAEB69
:100C600033FBC3EC33FCED33FD7E0A919E8B638A2C
:100C7000627896303A02789EE6FA7B007897E6FC36
:100C80007D007E00303A10C3EA33FAEB33FBC3EC4D
:100C900033FCED33FD7E0A919E8B618A6022C3ECAA
:100CA0009EFCED9400FDC3EC9AFCED9BFDC3EC941F
:100CB00023ED940050047C237D00C3EC94FFED945D
:100CC0000140047CFF7D017BFF0B7A000AEA70097A
:100CD000C3EC33FCED33FD81C9EC8AF0A4AEF0ED3A
:100CE0008AF0A42E947C40E4EAF460DD22D23691AE
:100CF0003812056D12056D7A007B007C10120565B7
:100D0000E5542AFA74003BFBDCF37C04C3EB13FBD1
:100D1000EA13FADCF7FFEB60027FFFC2369138225C
:100D200078A5E6F95403D2867002C286E9540CD243
:100D3000877002C287E95430D2967002C296E95495
:100D4000C07000227567007568007597DE7597ADF5
:100D50007581C043FF8075EF0675A900712F7580FE
:100D60003F75F1F075A4C075803F75D4FF75900094
:100D700075F27F75A57F75900075D57F75A6017595
:100D8000E34075E202C290C292C294120571D29100
:100D9000D293D295120561C291C293C295712FE48C
:100DA000F8F6D8FD713F1213AE789886647530015D
:100DB000C2AF12057551CC12056D51D212056D519D
:100DC000D812056DB120C2AF75670075680078FA5A
:100DD00079FA308507D9FBD8F7021C0071CA91381F
:100DE00078988664712F75E405758811758E047581
:100DF000890975C80475910475D84075D90875F7C7
:100E000081759E0375960275DA4275DB4275A821DD
:100E100075E69075B801759B80759D0075D10C7550
:100E2000BC5975BB1075E88075B201120561D2AF6F
:100E3000753C00C230120575C231C232C233C234B1
:100E4000755200755300752200120571C3E5229496
:100E50000A5002E11DD231752200120571C3E5224C
:100E6000940A5002E11DC231D2327522001205717E
:100E7000C3E522940A5002E11D75E4D575885175C9
:100E80008E017589AA758C00758D00C2A9D2ABD26E
:100E9000AA756BC0756A14756E50C232D234752251
:100EA0000A120571756A10C3E522940A755200751D
:100EB00053004069758E0C756B80756A28756E28B5
:100EC00075220A120571756A20C3E522940A7552CB
:100ED000007553004047758E0C756BC0756A1475AC
:100EE0006E1475220A120571756A10C3E522940A00
:100EF000755200755300402575E405758811758E8F
:100F000004758909D2A9C2ABC2AAC234D2337522F0
:100F100000120571C3E522940A4002A1C6120565BC
:100F2000203003020DC6C2AF51CC51CC51CCD2AF50
:100F3000120575203403303A03020FDB1205657881
:100F40008CE6C394015002E1DBE530C3940150020A
:100F5000E1DB7567A57568F17F02D236913812051D
:100F600071C2AFC2369138C3E554947FD2AF406BA3
:100F7000120561C2AF51DED2AFDFDF91EDC3EF7872
:100F800097F612057512149B7F0AD2369138120516
:100F900071C2AFC2369138C3E554947FD2AF50E8E6
:100FA000120561C2AF51CC12056951CCD2AFDFDA64
:100FB00091EDEF24037896F6F87997E7C3942340F0
:100FC00003985006E824237897F61205751213F556
:100FD0001214CA1205719138020DC6756700756842
:100FE00000120571C3E55494014002E133C2AF51D0
:100FF000DE51DE51DED2AF120575753000E4F537F3
:10100000F5380537E537F4703F0538789AE67819F2
:10101000146012783214600D787D14600878FA1428
:101020006003753800C3E53898401D120B2F120578
:1010300061153875370078998664C2AF120ADED21E
:10104000AF78988664120571120569E52370030272
:101050000DC6C3E5549401500AC3E55294015016DD
:10106000021002120571E5237003020DC6755200CD
:10107000755300021218C3E55294017017C2AF12E3
:101080000B2F78998664120ACC78988664D2AF12B6
:101090000571410AC3E55294027017C2AF120B2FBB
:1010A00078998664120AD278988664D2AF12057154
:1010B000410AC3E55294037017C2AF120B2F7899FF
:1010C0008664120AD878988664D2AF120571410AF4
:1010D000C3E55294047017C2AF120B2F789986643F
:1010E000120ADE78988664D2AF120571410AC3E510
:1010F0005294057017C2AF120B2F78998664120AAA
:10110000DE78988664D2AF120571410AC3E5529425
:10111000077019C3E5539406500201527401303A26
:101120000274037888F6C238C239410AC3E5529482
:10113000087019C3E5539406500201527402303A04
:101140000274047888F6D238D239410AC3E5529441
:10115000097017C3E553940650020152303A0BC38D
:101160007888E69402F6C23A410AC3E552940A70BE
:1011700016C3E553940650020152203A0A7888E6D5
:101180002402F6D23A410AC3E55294147025C3E50D
:1011900053940650020152C2AF901A0B740093D2BE
:1011A000AF7888F613C238C2394002D2384002D232
:1011B000398057C3E55294157038C3E553940640FF
:1011C0004FC2AF901A0B740093D2AFF8B8010274FB
:1011D00002B802027401B803027404B80402740372
:1011E0007888F613C238C2394002D2384002D23968
:1011F0008018C3E552940C70117567A57568F1C32A
:10120000E5539406400A71F5D2AF7552007553004C
:101210007567007568000152C2AF120B2FE4D2AFA0
:10122000E4F55EF524F525F53D755E0812056112BD
:1012300005CA30EDFDA8BDA9BEE97001F8885F12AE
:1012400005CE755E08C2AF120635855D5B855D5CB7
:10125000D2AF303A07C238303502D238D228753989
:1012600000120A87120AAA12064412064B120644FA
:1012700012064B1206441208C21209B31209FB12DD
:10128000064B1208B2202C03120584302C031205E1
:10129000B41209B3120A1E12064B1208C21209B385
:1012A000120A4112064B1208B21209B3120A641252
:1012B000064B1208C21209B3120A8712064B120516
:1012C000CA1208B21209B3120AAA1205CE12064BAC
:1012D000302827855D5B79187A0CC3E53999400E73
:1012E000C228D2298A3B855D5B855D5C800CC3E5A5
:1012F0005494014003021276618030291F202B1C78
:10130000E53B147006C229D22A4176F53B203A0704
:10131000C3E554940140030212768064753C0020BA
:101320003A0F78FA79A4E760027803C3E55598503C
:101330004FE523604B303A17203805203507800FE2
:10134000303502800A202B07D22B855D5B41A678C1
:10135000F0302B05855D5B7820C3E548985003028B
:101360001276302B1BC22BC238303502D238D2292C
:10137000753B12855D5B4176053CE55460026183F7
:10138000753C00C2AF120B2F752400752500D2AF3B
:10139000120571120B2F78A4E66006D291D293D277
:1013A00095C3E53C94044003020DC6020FFD901A5C
:1013B0000D7820912EE520B4550AA3912EE520B496
:1013C000AA0280137567A57568F1120B3F71F57558
:1013D0006700756800801D901A0378807B0A912E43
:1013E000A308DBFA901A0F788C7B1A912EA308DBE6
:1013F000FA901A2922C2AF9171914E901A0074107E
:101400009133A374079133A374219133901A037815
:10141000807B0A9132A308DBFA901A0F788C7B1A32
:101420009132A308DBFA91849162901A2922E49305
:10143000F622E6438F01538FFDFFC3E583941C40E2
:101440000122EF8567B78568B7F0538FFE22438F7F
:1014500002438F018567B78568B7901A0DF0538FE7
:10146000FC22901A0D74559133901A0E74AA913380
:10147000227A3079D07820901A40912EE520F70911
:10148000A3DAF7227A3079D0901A40E7913309A392
:10149000DAF9227C05120575DCFB22C2AF120ACCF8
:1014A000120AD2120AD8120ADE120569120ACC12E6
:1014B0000AD2120AD8120ADE120569120ACC120ADE
:1014C000D2120AD8120ADED2AF22C2AF120ADE123C
:1014D0000AD8120AD2120ACC120569120ADE120ABE
:1014E000D8120AD2120ACC120569120ADE120AD8E0
:0914F000120AD2120ACCD2AF227A
:1019FD00020D44100721FFFFFFFFFFFF09FF01FF4D
:101A0D0055AA01FFFFFFFFFF03FFFFFF25D0285061
:0D1A1D0004FF02FF7AFF0701FFFF0000FF3A
:101A400023455F4C5F33302320202020202020209E
:101A500023424C48454C492445464D3842313023B9
:101A60002020202020202020202020202020202076
:101C0000C2AFC2D37597DE7597AD7581C075A90057
:101C100043FF80752438752503B1DB7529A5752A26
:101C2000F143F12053A4DFD28575D4FF75E3407DE5
:101C3000FA780379E67C10752200752300901DE880
:101C40007B0675249875250130850281482085081A
:101C5000D8FBD9F9DCF781BA308508D8FBD9F9DC93
:101C6000F781BAB19BE493A3C39A6004DDC381BA40
:101C7000DBDBB18D600281317B08E493FAA3B16EA6
:101C8000DBF87A30B16E752200752300B18DEAFC65
:101C9000EBFDC3ED94FE400EB18D8A278B28ED300D
:101CA000E0048A828B83B18D7AC270D8C3ED94FE32
:101CB000601950CEBD0029EC600F7520007521FF22
:101CC000752900752A000200008100A827A92808AC
:101CD00009D804D90281DDB191EAF281D10D81A642
:101CE000C3ED94035051EDA2E092007AC5C3E582A2
:101CF0009400E583941C508C200010438F02438F86
:101D0000018529B7852AB7F0300027A827A9280818
:101D100009438F01538FFDD804D902A132C3E58353
:101D2000941C4003A3A117E28529B7852AB7F0A325
:101D3000A117538FFC81827AC1BD030CE493A3FAEF
:101D4000B152DCF8B14A81828184AA22AB23B16E00
:101D5000EBFAEA6222752608C3E52313F523E52290
:101D600013F52250066323A0632201D526EAB1DBD6
:101D7000B1DB75260AEAF4200102D285300102C2E5
:101D800085B1DBC3134002C201D526EB22B191EA33
:101D9000FB208502A191308502A196752608AE240C
:101DA000AF25C3EF13FFEE13FEB1DFB1DBC3EA13C0
:101DB0003085024480FA30E703632201C3E5231330
:101DC000F523E52213F52250066323A0632201D5F3
:101DD00026D9E52265236523F52222AE24AF250E00
:101DE0000FDEFEDFFCD20122424C48656C693437BD
:061DF0003164E8B10601B8
:00000001FF
